:10000000B601AD290408A700861105120512831652
:10001000861105120512F030850583122708B618DF
:100020002F283A30A100983016213330A600442002
:100030001330A1008830162144206430152144205B
:10004000643015212230A600442028302E200C30A8
:100050002E2006302E20B61427082F283614A6008E
:10006000361C3D280512033C031C42284220073061
:10007000A100D0301621031408003614FE3C0319E9
:10008000A8290516A60E361C36108615F0308505F3
:1000900026080F3985048611A60E361844283230FA
:1000A000152103140800083037190130A300A201FC
:1000B0003A0884003808F0203808800484130005CA
:1000C000FF3E371DA20C3719A20D32301521A30BAC
:1000D0005A2822080314A829A20008303719013031
:1000E000A300A20C3A0884003808F020380803184E
:1000F00080043C30152138088004A30B71280314B8
:10010000A829B71CA8298728B700371CA8293A08AE
:1001100084003808F0200130A100F430162138089E
:1001200080040130A100F4301629B800EE200A3016
:1001300008213808800484138006A001A1018417D7
:100140003808800664008006841300050319AE2871
:100150002408A0070318A10F9F28A1032108A8299C
:10016000A40029080319A829A321A0002518831792
:1001700024088400200880008313A40AA903B1285E
:10018000B71329080319B7170530A8002730A300B3
:100190001030D6200330A300E830D620A30164300D
:1001A000D620A3010A30D6202408DD28A200250885
:1001B000A1002408A00071212008A000A8030319B1
:1001C000B71329080319E728280203180800200894
:1001D000031DB713B71B0800303EA3298004F32882
:1001E000FF3A8005F428FF3A84178005A829831672
:1001F0009B001C141A08A82983169A001C15553058
:100200009D00AA309D009C149C1804291C11A8294B
:10021000A301A200FF30A207031CA307031CA82907
:100220000330A100DF3016210A29A101E83EA00019
:10023000A109FC30031C1F29A00703181C29A007D3
:100240006400A10F1C2920182529A01C29290000C1
:10025000292908000310A10CA00CFF3E03182A292D
:100260002008A829A101A301A20002304829A20068
:1002700003304829A101A301A20001304829A301AC
:10028000A20006304829A101A301A2000430482998
:10029000A80023082102031D4F2922082002043050
:1002A00003180130031902302805031DFF30A82967
:1002B0000038031DFF300405031DFF30A829040486
:1002C000031DFF30A829A2002008A6002408A000D2
:1002D0002608A4002108A6002508A1002608A500DC
:1002E0007329A501A4011030A600210DA40DA50DB0
:1002F0002208A4022308031C230FA5020318872940
:100300002208A40723080318230FA5070310A00D34
:10031000A10DA60B75292008A8291030A800A1015D
:10032000A001A70CA60C031C9B292208A0072308E8
:100330000318230FA107A10CA00CA50CA40CA80B5B
:1003400091292408A829840031088A0030088200F5
:100350008313031383126400080007309F00831681
:100360003030860085018312F430D4000130D5008E
:100370006430E000F430CC000130CD009F2D063019
:10038000BA008030B8000130842033306C208120E6
:100390000630BA008030B800003084200830A90050
:1003A0005330B000B101A5013C30B02081200800DD
:1003B0000630BA008030B8000130842055306C20FF
:1003C0003C086C203D086C203E086C203F086C20E7
:1003D00040086C2041086C2042086C2043086C20C7
:1003E00044306C2081200630BA008030B8000430E0
:1003F0008420532001390319E310031DE3148120E5
:100400006400E31CF3290630BA008030B8000130E4
:10041000842055306C203C086C203D086C203E0840
:100420006C203F086C2040086C2041086C2042087A
:100430006C2043086C20BE306C2081200630BA004E
:100440008030B800023084205320CE005320CF00EB
:1004500081200800D8217130A6000230A7004E0884
:10046000A2004F08A3008D21DE00A3010A30632102
:10047000D0002108D1006530A6000430A7004E0846
:10048000A2004F08A3008D21DE00F0304E05B2001F
:100490000F304F05B3003208A0003308A10004302C
:1004A0002D21D0002108D1000F304E05B200B3013C
:1004B0003208A6003308A7007130A2000230A30062
:1004C0008D21C6002508C700FE300320013003201F
:1004D00054300320653003206D300320703003203A
:1004E0003A30032020300320A9015008A40051080D
:1004F000A5000230B000B101C0202E300320A901B8
:100500004608A4004708A5000230B000B101C02091
:10051000DF3003204330032020300320080006147E
:100520008316061083120130A300903009210610B3
:1005300083160610831286148316861083120130E8
:10054000A3009030092186108316861083120615A9
:100550008316061183120130A30090300921061181
:1005600083160611831206178316061383120130B1
:10057000A300903009210613831606138312080086
:1005800006148316061083128614831686108312AF
:100590000615831606118312061783160613831297
:1005A0000800061083160610831286108316861024
:1005B000831206118316061183120613831606137F
:1005C00083120800831601309B0083126108FC200F
:1005D00008000130F720E1006108A000013043214C
:1005E000B2006108A00006303A21B400320884004D
:1005F00034085F21B400B5006400340835040319E1
:10060000042B0130E100E2220800D12206148316F7
:10061000061083120800D1228614831686108312D6
:100620000800D12206158316061183120800D12274
:1006300006178316061383120800052308000B23F0
:10064000080011230800172308002330D600D70123
:100650006E30C400C501352B08001930D600D70113
:100660006430C400C501352B08004408DC00E401F7
:10067000E501DF01E201052341240130D800D90161
:100680005808A0005908A1005708A30056083C21AB
:10069000031DB72B640001305C02031C532B0614AE
:1006A000831606108312640001306402031C5C2B65
:1006B0008614831686108312640001306502031CC1
:1006C000652B0615831606118312640001305F0244
:1006D000031C6E2B0617831606138312C801C9016B
:1006E0004808A0004908A1004508A30044083C218F
:1006F000031DB32B5C08A000A1014908A300480812
:100700003721031D872B06108316061083126408F9
:10071000A000A1014908A30048083721031D942B1C
:1007200086108316861083126508A000A10149086F
:10073000A30048083721031DA12B061183160611BB
:1007400083125F08A000A1014908A30048083721CF
:10075000031DAE2B06138316061383120A25C80A3F
:100760000319C90F702BD80A0319D90F402BB923CD
:100770003D2B64006208003C031DC02BDC03E40A2F
:1007800064006208013C031DC72BE403E50A640012
:100790006208023C031DCE2BE503DF0A64006208F9
:1007A000033C031DD52BDF03DC0A6208A0000030E8
:1007B0003221B2004408A0004508A100640833219A
:1007C000B4003208840034085821B400B500640035
:1007D000340835040319F02B0130E2000B234124C7
:1007E0006208A00001303221B2004408A000450890
:1007F000A10065083321B400320884003408582170
:10080000B400B50064003408350403190B2C023021
:10081000E200112341246208A00002303221B2001C
:100820004408A0004508A1005F083321B400320845
:10083000840034085821B400B5006400340835043D
:100840000319262C0330E200172341246208A0007C
:1008500003303221B2004408A0004508A1005C0822
:100860003321B4003208840034085821B400B500A4
:100870006400340835040319402CE20105234124A7
:1008800008000130DA00DB015A08A0005B08A10073
:100890004D08A3004C083C21031D542C01300821B5
:1008A000DA0A0319DB0F442C080064006108013CDC
:1008B000031D672CFE300320C0300320423003208C
:1008C0006C3003207530032065300320EB2C64006E
:1008D0006108023C031D772CFE300320C03003204A
:1008E000523003206530032064300320EB2C640079
:1008F0006108033C031D8B2CFE300320C030032015
:1009000057300320683003206930032074300320FF
:1009100065300320EB2C64006108043C031D9F2C10
:10092000FE300320C0300320473003207230032004
:1009300065300320653003206E300320EB2C64000B
:100940006108053C031DC52CFE300320C030032088
:100950004330032079300320633003206C300320C0
:100960006530032020300320413003206C30032009
:100970006C30032020300320533003206C300320E0
:100980006F30032077300320EB2C64006108063CB5
:10099000031DEB2CFE300320C03003204330032026
:1009A00079300320633003206C300320653003204E
:1009B00020300320413003206C3003206C300320B2
:1009C00020300320463003206130032073300320A1
:1009D00074300320EB2C0800640007306102031C14
:1009E000F42C0130E100F52CE10A0A30082108005E
:1009F000D20A0319D30A5208A0005308A1005508CF
:100A0000A30054084521031D092D2A225524D20193
:100A1000D30108006400061A0E2DDD010030061A0D
:100A20000130A00001303221B2005D08A00000308A
:100A30003221B4003208840034085821B400B500D3
:100A40006400340835040319262D282DF8240800E5
:100A50006400061A2C2DDD010030061A0130A000BA
:100A600001303221B2005D08A00000303221B40014
:100A70003208840034085821B400B50064003408FA
:100A800035040319472D0130DD00EC2455246400A2
:100A90006108013C031D4D2D1D2364006108023CCB
:100AA000031D532D1F2364006108033C031D592DB2
:100AB000212364006108043C031D5F2D232364008F
:100AC0006108053C031D652D252B64006108063C6B
:100AD000031D6B2D2D2BF824282D2A22B430A400C1
:100AE0000630840020309520CA00CB01FE30032060
:100AF000C03003204C3003206930032067300320CE
:100B000068300320743003203A3003202030032063
:100B1000A9014A08A4004B08A5000230B000B101A9
:100B2000C0204A08A0004B08A10060083F21031D17
:100B30009B2DC0229C2DD1220A3008216D2D013021
:100B4000A300F4300921BF216400061EA82D6D2DDD
:0C0B5000DD01E922D201D3015524282D3B
:02400E00553F1C
:00000001FF
